:030000000219FDE5
:03000B000200AA46
:03002B0002015679
:03005B000202E8B6
:030073000202D5B1
:1000800002030406080C10182030406080040608A3
:100090000C10182030406080A0C00003070F1F0D17
:1000A0000D04050D050205030302C2AFC0D0C0E078
:1000B000206214E5256009E473E525F4F58AD2622F
:1000C000D0E0D0D0D2AF3285268AC262E526F46075
:1000D00029D0E0D0D0C293C295C297D2AF32C2939A
:1000E000C295C297206F0C206609740ED5E0FDE51D
:1000F0007B4290D0E0D0D0D2AF32758A00C28DD290
:100100006201F301B9306805206602D29301B9306B
:100110006805206602D29501B9306805206602D2D2
:100120009701B9C29230680A206607740CD5E0FDC9
:10013000D29301B9C29430680A206607740CD5E0E6
:10014000FDD29501B9C29630680A206607740CD5B5
:10015000E0FDD29701B9C2AFC2AD53E6EFC0D0C047
:10016000E0D2D3D2AFC2CEE52A6007207449152A67
:1001700021B77800790020742EE580307E01F430BC
:10018000E30278FF53DACF207E0343DA20307E0388
:1001900043DA10C2D8C271E580307E01F430E30248
:1001A00079FFC3E89970CB306103752A1820740376
:1001B000752A18885CD27020740DE52B6004152B0D
:1001C00021C743DA01C2D82070024136A85C206101
:1001D00002C2702074367982B70431C3E894F040CB
:1001E0000374F0F8E8C4540F28F87984B703024187
:1001F0000CC313C3138721200802C313200A06C3AC
:10020000C898F8410C28F8500374FFF88822E52DAF
:1002100054066022206B1FE536C333C333F8E56410
:10022000C313C313F9C3952240028922E82522F59E
:100230002250037522FF7882B6044E852224A8241A
:10024000C3E52495614002A861C3E895634002A814
:10025000638825E56670024187C3E8AA669A500361
:10026000E8FAE4F9EAC333FBE568F45B29400D25BD
:1002700067F8E56760021567400B41870AC3E567C9
:100280009A5002056778FF8826C3E525944040020E
:10029000D26420CF0AD0E0D0D043E610D2AD32C233
:1002A000CF053A7801E52A6005307402152AC3E5C6
:1002B0005C94014005755F0041CB75600075690075
:1002C000E55F2401F55F5003755FFFD0E0D0D043B8
:1002D000E610D2AD32C2AF53E67F7592FA7593FF46
:1002E000C260759104D2AF32C2AF53E6EFC2ADC067
:1002F000D0C0E0C0F0D2D3D2AFA8FBA9FCC2D830A6
:100300007102614F53DACF207E0343DA10307E034F
:1003100043DA20D271E580307E01F420E3026126C9
:1003200088278928A17C53DACF207E0343DA203046
:100330007E0343DA10C2D8C271307402A16878001B
:10034000E580307E01F430E302A168885CA150535F
:10035000DACF207E0343DA20307E0343DA10C27105
:10036000206102812853DACF207E0343DA10307EE9
:100370000343DA20C2D8D27188578958C3E895550B
:10038000F8E99556F97B007E087A00C3E8948CE979
:1003900094005005755B00811A882178A2E6A82197
:1003A0006055C3E894C8E994005008E4D2E4FB7AAD
:1003B0000A61F5C3E89468E994015008E4D2E3FBCC
:1003C0007A0F61F5C3E894D0E994025008E4D2E2D0
:1003D000FB7A1E61F5C3E894A0E994055008E4D2C5
:1003E000E1FB7A3C61F5C3E89498E994085008E48D
:1003F000D2E0FB7A787E00C3E89559FCE9955AFD76
:1004000030E70AECF42401FCEDF43400FD755B00E8
:10041000C3EC9AED9E5003755B018859895A855744
:10042000558558567802A150C3E89527F8E99528D4
:10043000F9307C02A134307B02A134307A02A12D44
:10044000207502814BE9FDE8FC816AE9C313F9E8F4
:1004500013F8307902A12DE9C313F9E813F83078C5
:1004600002A12DE9C313FDE813FC20612CC3EC9419
:0F0470001CED940240028181ED701EC3EC94C814
:10047F0050180529E52970021529C3E529940A505A
:10048F0002A168755C00D270A168E5296002152988
:10049F007888E6F97400207F087896B90302789E71
:1004AF00E624FAFEE43400FFC3EC9EFCED9FFD92C0
:1004BF0008B90310A2085007207609D27681D330ED
:1004CF007602C276A2085016B9030DECF42401FC93
:1004DF00EDF43400FD0204ED78007900A134B90386
:1004EF0015EC33FCED33FDC3EC940AFCED9400FDE9
:1004FF0050047C007D00C3EC94FFED94004006781F
:10050F00FF7900A134EC8572F0A4C5F0A2F733F89F
:10051F007900400302055078FF7900020550E9C3C6
:10052F0013F9E813F8307C0EE9600278FFC3E81383
:10053F0038F8E43400F9C3E894FFE99400400278F6
:10054F00FF885CD270206102A168741FF4552F4B95
:10055F00F52FC274EB7002D274752A1830740375BC
:10056F002A0A306102A17C20740353DAFE2074033F
:10057F00752B06D0F0D0E0D0D0D2AD43E610327953
:10058F00010205AC79030205AC790A0205AC791EAC
:10059F000205AC79640205AC79C80205AC7817E4A2
:1005AF00D5E0FDD8FAD9F6227A147B780205D37AF2
:1005BF00107B8C0205D37A0D7BB40205D37A0B7BAB
:1005CF00C80205D37902E4C294D5E0FDD295D5E0F7
:1005DF00FDC295D5E0FDD294D5E0FDE920E002D231
:1005EF009330E002D297E573D5E0FDE920E002C237
:1005FF009330E002C2977496D5E0FDD9C9EAF8D5D9
:10060F00E0FDD8FBDBBEC29422C37C007D0075F0F9
:10061F000005F0EA33FAEB33FB50F6EB13FBEA136A
:10062F00FAC3E9FFE8FEE89AF8E99BF95004EFF9FD
:10063F00EEF8B3EC33FCED33FDD5F0DFEDF9ECF86C
:10064F0022E889F08A20D2D4F8A9F07B0030F70B8A
:10065F007BFFF42401F8E9F43400F9E88520F0A4D5
:10066F00ADF0F8E98520F0A4AFF0FEED2EF974009F
:10067F003FFA7C04C3EA13FAE913F9E813F8DCF440
:10068F008BF030F70AE8F42401F8E9F43400F9E8C4
:10069F0089F0C2D4F8A9F0227882B60403020702C7
:1006AF00C3E55C940140030206CC852224E4F544A3
:1006BF00F545F546F547F548C26E0207027882E622
:1006CF00FCD26EE522F523783879C7AA40AB41C337
:1006DF00EB13FBEA13FAEC146013C3EB13FBEA13EF
:1006EF00FAEC14146007C3EB13FBEA13FAD1188862
:1006FF0044894522C3E5449523F8E5459400F95014
:10070F000CC3E89480E994FF4016020733C3E894C2
:10071F007FE994005003020733787F790002073393
:10072F00788079FF8849894A22E5492546F8E54AC4
:10073F003547F9854A20E4300701F43548FA30E7A8
:10074F0009C3EA94F04015020771C3EA940F5003EE
:10075F0002077178FF79FF7A0F020771780079002D
:10076F007AF0C3E5249561500AC374019524500BA8
:10077F0002078FE54A20E70E02078FE54A30E706AA
:10078F00884689478A482278A5E6FAC3E54933F8AF
:10079F00E54A33F9D150E930E70BC3E89480E99487
:1007AF00FF4013E1C9C3E8947FE994005002E1C907
:1007BF00787F7900E1C9788079FFE820E715C3E5F4
:1007CF002398F84009C3E8940140030207F0780129
:1007DF000207F0E8F424012523F840030207F0781C
:1007EF00FF884B2278A6E6FAA847A948D150E930EE
:1007FF00E70CC3E89401E994FF4016020824C3E80C
:10080F0094FFE99400500302082478FF790002084E
:10081F0024780179FFE920E715C3E54B98F84009E3
:10082F00C3E89401400302084B780102084BE8F437
:10083F002401254BF8400302084B78FF88242278C7
:10084F00FFC26420693D206A12D264C3E541940A55
:10085F004009C3E52594405002C26479A1E76023A3
:0D086F00E541601F74FF8541F0848539F07C
:10087C00306A0375F005A4F8C5F0600278FFC3E890
:10088C0095645002A864886322C3E5409440E54116
:10089C009401E56350031401A6046002F56322027F
:1008AC0008AE2275E890227883E6FFE5E820ECF7A5
:1008BC00A8BDA9BE0570C3E57094084052757000C0
:1008CC00E9FA79A0E76044EA7007E571601B020859
:1008DC00E9C3E895716010E5715006600C140208CC
:1008EC00F50460F90208F5E571F571C394A8401B95
:1008FC007561C0C394054013756180C39405400BAA
:10090C00756140C39405400375610075BB0122E518
:10091C00612410500274FFF5617982B70402214200
:10092C00C3A861E524985002A824C3E8956340024B
:10093C00A86388258826E570B4070375BB1E22744E
:10094C003279A787F0A4C5F0A2F733F8C3E8956114
:10095C004002A8618822882488258826886422750C
:10096C0040007541F022C2AF75C820A8CCA9CDAA11
:10097C003A30CF010A75C824D2AFAB3BAC3C883BB4
:10098C00893CC3E89BF8E99C206908F9306702416F
:10099C007E21DBAD3D8A3DF9EA9DFA600478FF7952
:1009AC00FFAE3EAF3F8B3E8C3FA83BA93CC3E89EBD
:1009BC00F8E99FF9C3E54113FBE54013FAE82AF582
:1009CC0040E93BF54150067540FF7541FF4125AAB2
:1009DC0040AB41AC40AD417E047F02C3EB9404407C
:1009EC00021E1FC3EB940840021E1FC3ED13FDEC47
:1009FC0013FCDEF7C3EA9CFAEB9DFBEF6009C3E93D
:100A0C0013F9E813F8DFF7EA28FAEB39FB8A408B85
:100A1C004150067BFF8B408B41C3EB94025002D2BA
:100A2C00673069047F0341507892E6FFC3E5379441
:100A3C008240110FC3E53794A040010FC3EF940619
:100A4C0040027F057E02E541C4540FF9E541C454D0
:100A5C00F0F8E540C4540F28F8C3E89EFAE9940076
:100A6C00FB4009C3EA9402EB940050047A02E4FBC5
:100A7C0041CAAA40AB41EBC4FEEAC4540F4EFCC3BE
:100A8C00EA9CFAEB9400FBC3E813C313F8EA28FAC8
:100A9C00EB3400FB8A408B41C3EB94024002C267EB
:100AAC007802EBC4FE7B00EAC4540F4EFAC3EA98FA
:100ABC00FA4005C3940250027A027892E6FF306045
:100ACC000241CA855192855293D26043E680C3E4B9
:100ADC009AF8E49BF93067026156E8FAE9FBD3E92E
:100AEC0013FDE813FC88518952C3EF94036038EF6F
:100AFC0020E00DE82CF8E93DF9ECFAEDFB020B1FB8
:100B0C00E828F8E939F9C3E82402F8E93400F97A5D
:100B1C00FE7BFFC3EF9403400E8A538B54884D89A0
:100B2C004E8C4F8D50618A885389548A4D8B4E8CD4
:100B3C004F8D503069127553F07554FF754FF07529
:100B4C0050FF7551F07552FF618AE8FAD3E813FC37
:100B5C008851C3EF94036020EF20E007E82CF8ECF9
:100B6C00FA6176E8282402F87AFEC3EF9403400871
:100B7C008A53884D8C4F618A88538A4D8C4FE56817
:100B8C00C3335002646BF5683060026194753402B3
:100B9C00D26043E680E52D54066034A840A941C3D9
:100BAC00E913F9E813F8C3E913F9E813F830690409
:100BBC00E92440F9C2AF53E67F759100C3E498F580
:100BCC0094E499F595759104D26043E680D2AF22F6
:100BDC00D265754300752000306C03752040020B04
:100BEC00FBD265754300752040306C03752000788E
:100BFC00017901206720E52D54066002C265791445
:100C0C00E541C313700104F8C39414400278143006
:100C1C006904781B791B206010E543600C30690374
:100C2C00D53404D26D81A6719C0543E59E7005E513
:100C3C009B020C42E59A5440B52002819030690920
:100C4C0008C3E899400118812220650A08C3E89975
:100C5C00400261FB8122C265C2AF53E67F759100F1
:0E0C6C003067127594007595FE759104D26084
:100C7A0043E680D2AF61FBAE40AF41C3E49EF59438
:100C8A00E49FF5958175C3E5339401500261FB3009
:100C9A00650261FBD80281A48122C26DC2AF53E60C
:100CAA007F759100855394855495759104854D926D
:100CBA00854E93D26043E680D2AFE52D5406600894
:100CCA00206A020533020CE2306D0D206C0A2065A1
:100CDA00071581158102158F227800306405306569
:100CEA00027801E53775F007A4F9E5F028F5F0E98F
:100CFA00A2F013A2F113A2F213F537C394785003AA
:100D0A00753778C3E53795384008D266C293C295DD
:100D1A00C297306002A11C854F92855093D26043DE
:100D2A00E68022207D19C2AF754202C294D2923067
:100D3A006202D297D2AF759F33759E00020F2EC200
:100D4A00AF754202C294D296306202D293D2AF7584
:100D5A009F33759E00020F2E307243207D20C2AF52
:100D6A00754203900134757B10C297C296306204B3
:100D7A00D295A180D294D2AF759E23020F2EC2AF14
:100D8A00754203900134757B10C293C2923062049B
:100D9A00D295A1A0D294D2AF759E22020F2E207DA9
:100DAA0017C2AF75420390010FC297306202D29503
:100DBA00D2AF759E23020F2EC2AF75420390010F68
:100DCA00C293306202D295D2AF759E22020F2E20B4
:100DDA007D16C2AF754204C292D296306202D29593
:100DEA00D2AF759E22020F2EC2AF754204C296D2AE
:100DFA0092306202D295D2AF759E23020F2E3072C4
:100E0A0049207D23C2AF754205900123757B04C238
:100E1A0095C294306204D293C126D292D2AF759F02
:100E2A0033759E00020F2EC2AF75420590014575BB
:100E3A007B40C295C294306204D297C149D296D2FD
:100E4A00AF759F33759E00020F2E207D1AC2AF75B3
:100E5A004205900105C295306202D293D2AF759FC6
:100E6A0033759E00020F2EC2AF754205900119C25A
:100E7A00953062E8D297D2AF759F33759E00020F04
:100E8A002E207D16C2AF754206C296D294306202F7
:100E9A00D293D2AF759E23020F2EC2AF754206C2FD
:100EAA0092D294306202D297D2AF759E22020F2E4E
:100EBA00307243207D20C2AF754201900145757B97
:100ECA0040C293C292306204D297C1D8D296D2AFAE
:100EDA00759E22020F2EC2AF754201900123757BC7
:100EEA0004C297C296306204D293C1F8D292D2AFAA
:100EFA00759E23020F2E207D17C2AF754201900105
:100F0A0019C293306202D297D2AF759E22020F2E77
:100F1A00C2AF754201900105C297306202D293D2E4
:100F2A00AF759E23C26622900103757B00C293C2ED
:100F3A0095C297C292C294C296C2622278807609FA
:100F4A000876090876040876FF0876030876FF080B
:100F5A007607087601087601087601788C7601080A
:100F6A0076FF0876FF0876FF0876FF0876FF087690
:100F7A00030876FF0876FF0876FF0876250876D0FC
:100F8A000876280876500876040876FF087602085C
:100F9A00760008767A0876FF0876010876010876E0
:100FAA0000087603087600227887E6FFC2727888FE
:100FBA00E6C394036008C27DE630E102D27DC27EB8
:100FCA007889E630E102D27EC3EF94026008758E1A
:100FDA0001D273020FE5758E00C273227880E6147F
:100FEA009000809378A5F67881E614900080937833
:100FFA00A6F67886E61490008D9378A7F67886E6AA
:10100A00F539C394025003753902789CE67538FFA6
:10101A00B402037538A0B4030375388278A3E614C2
:10102A0090009A93F566120F3122227896E6FA78A2
:10103A0097E6FB7888E6B40305C3EB940EFB307F92
:10104A00047A007BFFC3EB9AFCC3948250027C8231
:10105A007572000572EC8572F0A4C3E5F0947D40C8
:0F106A00F222D27F113512059D7A007B007C1097
:10107900120593E55C2AFA74003BFBDCF37C04C39C
:10108900EB13FBEA13FADCF7FEC27F113522E5EF19
:1010990020E6037520000520903DFFE52014600639
:1010A900901FFF1460009304600375EF1253D9BFBA
:1010B9007581C043FF8012058E75EF0243B203E5C7
:1010C900B3240220E70DF521E5B120E0068521B31F
:1010D90043B101120F317580FF75A40075F1FE75DA
:1010E900D4F775900275A5FC75F2FC75D50075A04D
:1010F900FD75A60275F30275D60075B0FF75A701D7
:1011090075F4FF75E241120F31E4F8F6D8FD756800
:1011190001120F461215E078988673753001C2AF37
:101129001205A71205B712059D1205BE12059D12DB
:1011390005C512059DC2AF78FA79FA308307D9FB44
:10114900D8F7021C00120FB2120FE61134113578CC
:10115900988673120F3175881075890275C82475C0
:10116900910475D84075A82275B80275E690759BEB
:1011790080759D00759A80759C0075D10E75BC5857
:1011890075BB0175BA1F75E88012058ED2AF1208BA
:10119900AB75360053DACF207E0343DA20307E0365
:1011A90043DA1043DA01C2D8C2711205A7D2617BB2
:1011B900037A0CE55B70077A0CDB0302113E12051A
:1011C9009D20700302113EC270E55CC3940240E1A8
:1011D900E52F541F855E5DF55EB55DD5DAD5C26133
:1011E90053DACF207E0343DA20307E0343DA10C27C
:1011F900D8C27178A2E67008D274E52F54E0F52FB1
:10120900C2757529001205A2307409C3E529940A2B
:101219004002D27512059378023074027800C3E552
:101229005C9840F0C2AF1205B71205B71205B7D2E4
:10123900AF1205A7754C007888E6B40302611C1249
:101249000593788CE6C39401500302131CE530C35F
:101259009401500302131C207435C3E55C94FF50BC
:101269000302131CC2AF1205CCD2AF1205A2C3E50B
:101279005C940150EFC2AF1205B71205981205B779
:10128900D2AF1205A2C3E55C94FF40E90217887F3B
:1012990002D27F11351205A2C2AFC27F1135AE5CF1
:1012A900C3E55C947FD2AF407412058EC2AF1205BC
:1012B900CCD2AFDFDC116CC3EE7897F61205A7121A
:1012C900162212170B7F0AD27F11351205A2C2AF5F
:1012D900C27F1135AE5CC3E55C947FD2AF50E61294
:1012E900058EC2AF1205B71205981205B7D2AFDF46
:1012F900D6116CEE24037896F61205A7121622125F
:10130900173A1205A21135C3E55C94FF50024160FA
:10131900021788C3E55C954C4003855C4C1205A215
:1013290078017988E7B403027805C3E55C9840023F
:101339004140C2AF1205CC1205CC1205CCD2AF1276
:1013490005A7753000E4F531F5320531E531F47062
:101359003F0532789AE67819146012783214600DD4
:10136900787D14600878FA146003753200C3E53299
:1013790098401D120F3112058E153275310078997A
:101389008673C2AF1205CCD2AF789886731205A2C4
:10139900120598E52A7005307402213E78012074FF
:1013A900027806C3E55C9840A17888E6C394036097
:1013B900031205A2E52A700302113EC2AF120F31D2
:1013C900E4F522F523F524F525F526F567D2AF785E
:1013D90085E6C333F565E4F544F545F546F547F586
:1013E90048F570F52CF52DF53775700875BB1E128B
:1013F900058E1208AFE5E820ECFBA8BDA9BEE9708F
:1014090001F888711208B375700875BB1E120FB206
:10141900C2AF7561FF12094B85226185226285225F
:1014290063D2AF75220175240175250175260185E1
:101439006069756A017888E6B40307C27D3076026F
:10144900D27DD268D269753300120E8B120EBA1290
:10145900096B12097212096B12097212096B120BCC
:0D146900ED1206A7120CE3120D2D120972F0
:10147600120BDC306E0312070320670312084E308E
:101486006703120895120CE3120D62120972120B11
:10149600ED306E03120738120CE3120DD9120972E1
:1014A600120BDC306E03120796120CE3120E0812B2
:1014B6000972120BED306E031207F3120CE3120ED3
:1014C6008B1209721208AF120BDC120CE3120EBA61
:1014D6001208B312097230693285646185646285C7
:1014E6006069756A0179187A0CC3E53399400FC2B1
:1014F60069D26A8A35856461856463021511C3E51C
:101506005C94014003021467021597306A1D206C33
:101516001AE535147006C26AD26B8167F535C3E5E4
:101526005C9401400302146702159775360078FA39
:1015360079A4E760027803C3E55F985054307404D9
:10154600E52A604D7888E6B40317207D05207607E6
:10155600A167307602A167206C07D26C8564618131
:10156600A678F0306C058564617820C3E541985013
:10157600028167306C1BC26CC27D307602D27DD28E
:101586006A75351285646181670536E55C6002A17E
:101596009A753600C2AF120F317887E6FE760212D0
:1015A6000FB27887EEF6E4F522F523F524F525F556
:1015B60026F565752C00752D00D2AF1205A2120F07
:1015C6003178A4E66006D293D295D297307409C3D7
:1015D600E53694044002213E614E901A0D782012A1
:1015E6001664E520B4550CA3121664E520B4AA03CC
:1015F600021602120F46121622021621901A0378BC
:10160600807B0A121664A308DBF9901A0F788C7B8C
:1016160019121664A308DBF9901A2822C2AF121613
:10162600A312167D901A00740E121669A374061280
:101636001669A37415121669901A0378807B0A122C
:101646001668A308DBF9901A0F788C7B19121668B6
:10165600A308DBF91216B6121694901A2822E49300
:10166600F622E6438F01538FFD75EF0275B7A57518
:10167600B7F1F0538FFE22438F02438F0175EF02BD
:1016860075B7A575B7F1901A0DF0538FFC22901A15
:101696000D7455D169901A0E74AAD169227A3079DF
:1016A600D07820901A40D164E520F709A3DAF72212
:1016B6007A3079D0901A40E7D16909A3DAF922ABDA
:1016C60074A875BB01027980BB02027981BB030253
:1016D6007982BB04027984BB05027986BB0602794E
:1016E60092BB07027987BB080279A3BB0902799CE2
:1016F600BB0A027988BB0B027989E8F7227C0512BE
:1017060005A7DCFB22C2AF1205B71205BE1205C53E
:101716001205CC1205981205B71205BE1205C512A0
:1017260005CC1205981205B71205BE1205C512059D
:10173600CCD2AF22C2AF1205CC1205C51205BE121D
:1017460005B71205981205CC1205C51205BE12057D
:10175600B71205981205CC1205C51205BE1205B7BB
:10176600D2AF22AE74AF75C2AF1205B71205B7126B
:1017760005B7120598DEF21205CC120598DFF8D2ED
:10178600AF22F10BF103F1037574017575017576DE
:1017960000F1697C05AD5C1205A7C3ED955C70F59B
:1017A600C3E55C9401400AC3E55C94FF403202172E
:1017B600C4D1C5D122F10BC2AF75EF12F103DCD54E
:1017C6000576C3E5769403500280C6F1030575E5F8
:1017D600741490009F93F808C3E57598500280AE84
:1017E600F103F1030574C3E574940C5002809C1256
:0C17F6000F46D122C2AF75EF121217038C
:0319FD000210973E
:101A00000E0615090904FF03FF0701010155AA018C
:101A1000FFFFFFFFFF03FFFFFF25D0285004FF0259
:091A2000007AFF0101000300FF40
:101A4000235467794B4631323041485623202020B9
:101A500023424C48454C4923463331302320202033
:101A60002020202020202020202020202020202076
:101C0000C2AFC2D353D9BF7581C043B20343FF8073
:101C1000752438752503B1C975EF0275E24043F1AB
:101C20000853A4F775D4FFD2837DFA780379E67C54
:101C300010752200752300901DD67B0675249875BB
:101C400025013083028142208308D8FBD9F9DCF7D3
:101C500081B4308308D8FBD9F9DCF781B4B189E4C9
:101C600093A3C39A6004DDC381B4DBDBB17B600264
:101C7000812B7B08E493FAA3B15CDBF87A30B15C8A
:101C8000752200752300B17BEAFCEBFDC3ED94FEE9
:101C9000400EB17B8A278B28ED30E0048A828B834B
:101CA000B17B7AC270D8C3ED94FE601350CEBD00F4
:101CB00025EC60097520007521FF0200008100A855
:101CC00027A9280809D804D90281D3B17FEA89AAB3
:101CD000F281C50D81A0C3ED94035049EDA2E092BD
:101CE000007AC5C3E5829400E583941C50902000DF
:101CF00010438F02438F0175B7A575B7F1F030001F
:101D00001FA827A9280809438F01538FFDD804D99C
:101D100002A12089AAE275B7A575B7F1F0A3A10DBC
:101D2000538FFC817C7AC1BD030CE493A3FAB140CC
:101D3000DCF8B138817C817EAA22AB23B15CEBFA5E
:101D4000EA6222752608C3E52313F523E52213F57D
:101D50002250066323A0632201D526EAB1C9B1C986
:101D600075260AEAF4200102D283300102C283B14F
:101D7000C9C3134002C201D526EB22B17FEAFB2082
:101D80008302A17F308302A184752608AE24AF258B
:101D9000C3EF13FFEE13FEB1CDB1C9C3EA13308315
:101DA000024480FA30E703632201C3E52313F523DD
:101DB000E52213F52250066323A0632201D526D91C
:101DC000E52265236523F52222AE24AF250E0FDE22
:101DD000FEDFFCD20122424C48656C693437316326
:041DE000F3100601F5
:00000001FF
